S12301007E012C486561646572203D200420416C6C6F63203D20042020526F6F74203D2079
S10B0120044572726F722004A1
S123012CBDC02186F09702BD202827037E02717F01287F01297F012A7F012BCE0103BDC0ED
S123014C09CE012ABDC015BDC021BD027DCE1000864DB710008643B710018646B7100286FD
S123016C53B710038602B71004CE0000FF1005CEFFFFFF1007CE5555FF1009CE0001FF10CD
S123018C2BCE0080FF102DCE0081FF102FCE0088FF1031CE1000BD201427037E0271CE01BE
S12301AC0DBDC0097C012BCE012ABDC015BD027D5FCE1000C18A22066C00085C20F6CE10B9
S12301CC00BD2014BD027D7C012B5FC17D2211CE1000BD201427037E02717C012B5C20EB71
S12301EC862DBDC0038620BDC003CE012ABDC015BDC021CE0117BDC0097C012BCE012ABDA3
S123020CC015BD027DCE1000BD20147C012BCE1000BD20147C012BCE1000BD20147C012B58
S123022CCE1000BD20147C012BCE1000BD20147C012BCE1000BD20147C012BCE1000BD208E
S123024C147C012BCE1000BD201427037E0271862DBDC0038620BDC003CE012ABDC015BD47
S122026CC0217EC000CE0121BDC009BDC0217EC000CE10008C120022056F000820F63995
S1232000BD204ABD20638601B79FD28620B79FD77E208039BD204ABD20638601B79FD286E0
S123202030B79FD77E209A39BD202FBD2054398604B79FD7BD204A86E0B79FD68601B79F0B
S1232040D186EFB79FD7BD204A39B69FD78480810026F739B69FD7840181002704B69FD11F
S1232060394F39B6012BB79FD3B6012AB79FD4B60129B79FD5B60128840F8AE0B79FD63939
S1232080BD204AB69FD784088108260CB69FD0A70008BD205427E9394F39BD204AB69FD779
S11720A084088108260CA600B79FD008BD205427E9394F390B
S9030000FC
